 lcdcbacklight

 Timestamp is 4da293c6 (Mon Apr 11 17:38:14 2011)

 Preferred load address is 10000000

 Start         Length     Name                   Class
 0001:00000000 00000004H .CRT$XCA                CODE
 0001:00000004 00000004H .CRT$XCZ                CODE
 0001:00000008 00000004H .CRT$XIA                CODE
 0001:0000000c 00000004H .CRT$XIZ                CODE
 0001:00000010 00000004H .CRT$XPA                CODE
 0001:00000014 00000004H .CRT$XPZ                CODE
 0001:00000018 00000004H .CRT$XTA                CODE
 0001:0000001c 00000004H .CRT$XTZ                CODE
 0001:00000020 00000282H .rdata                  CODE
 0001:000002a4 0000002aH .rdata$debug            CODE
 0001:000002d0 00001194H .text                   CODE
 0001:00001464 00000004H .xdata                  CODE
 0001:00001468 0000003cH .idata$2                CODE
 0001:000014a4 00000014H .idata$3                CODE
 0001:000014b8 00000098H .idata$4                CODE
 0001:00001550 00000078H .idata$6                CODE
 0001:000015d0 00000105H .edata                  CODE
 0002:00000000 00000098H .idata$5                DATA
 0002:00000098 0000009cH .data                   DATA
 0002:00000134 0000009cH .bss                    DATA
 0003:00000000 000000e0H .pdata                  DATA

  Address         Publics by Value              Rva+Base       Lib:Object

 0000:00000000       ___safe_se_handler_table   00000000     <absolute>
 0000:00000000       ___safe_se_handler_count   00000000     <absolute>
 0001:00000000       __xc_a                     10001000     corelib0:crt0init.obj
 0001:00000004       __xc_z                     10001004     corelib0:crt0init.obj
 0001:00000008       __xi_a                     10001008     corelib0:crt0init.obj
 0001:0000000c       __xi_z                     1000100c     corelib0:crt0init.obj
 0001:00000010       __xp_a                     10001010     corelib0:crt0init.obj
 0001:00000014       __xp_z                     10001014     corelib0:crt0init.obj
 0001:00000018       __xt_a                     10001018     corelib0:crt0init.obj
 0001:0000001c       __xt_z                     1000101c     corelib0:crt0init.obj
 0001:0000003c       ??_C@_19OBGHODPD@?$AAM?$AAo?$AAd?$AAe?$AA?$AA@ 1000103c     bspbacklight.obj
 0001:00000048       ??_C@_1CK@ENPFCICM@?$AAD?$AAr?$AAi?$AAv?$AAe?$AAr?$AAs?$AA?2?$AAD?$AAi?$AAs?$AAp?$AAl?$AAa?$AAy?$AA?2?$AAL?$AAC?$AAD?$AAC?$AA?$AA@ 10001048     bspbacklight.obj
 0001:00000074       ??_C@_1CM@JBPFNDBJ@?$AAD?$AAr?$AAi?$AAv?$AAe?$AAr?$AAs?$AA?2?$AAB?$AAu?$AAi?$AAl?$AAt?$AAI?$AAn?$AA?2?$AAL?$AAC?$AAD?$AAA?$AAD?$AA?$AA@ 10001074     bspbacklight.obj
 0001:000000a0       ??_C@_1CC@OPDEBLKM@?$AAA?$AAC?$AAB?$AAa?$AAc?$AAk?$AAl?$AAi?$AAg?$AAh?$AAt?$AAL?$AAe?$AAv?$AAe?$AAl?$AA?$AA@ 100010a0     backlight_common_topaz_v1:backlight.obj
 0001:000000c4       ??_C@_1CG@LFMPNLPM@?$AAB?$AAa?$AAt?$AAt?$AAB?$AAa?$AAc?$AAk?$AAl?$AAi?$AAg?$AAh?$AAt?$AAL?$AAe?$AAv?$AAe?$AAl?$AA?$AA@ 100010c4     backlight_common_topaz_v1:backlight.obj
 0001:000000ec       ??_C@_1CO@MGKPHPG@?$AAC?$AAo?$AAn?$AAt?$AAr?$AAo?$AAl?$AAP?$AAa?$AAn?$AAe?$AAl?$AA?2?$AAB?$AAa?$AAc?$AAk?$AAl?$AAi?$AAg?$AAh?$AAt?$AA?$AA@ 100010ec     backlight_common_topaz_v1:backlight.obj
 0001:0000011c       ??_C@_1O@ILKHMLBG@?$AAU?$AAs?$AAe?$AAE?$AAx?$AAt?$AA?$AA@ 1000111c     backlight_common_topaz_v1:backlight.obj
 0001:0000012c       ??_C@_1BG@LEIIKALA@?$AAU?$AAs?$AAe?$AAB?$AAa?$AAt?$AAt?$AAe?$AAr?$AAy?$AA?$AA@ 1000112c     backlight_common_topaz_v1:backlight.obj
 0001:00000144       ??_C@_1BE@PJBHBNNG@?$AAA?$AAC?$AAT?$AAi?$AAm?$AAe?$AAo?$AAu?$AAt?$AA?$AA@ 10001144     backlight_common_topaz_v1:backlight.obj
 0001:00000158       ??_C@_1BO@PELGLPFE@?$AAB?$AAa?$AAt?$AAt?$AAe?$AAr?$AAy?$AAT?$AAi?$AAm?$AAe?$AAo?$AAu?$AAt?$AA?$AA@ 10001158     backlight_common_topaz_v1:backlight.obj
 0001:00000178       ??_C@_1DA@IKPIDNLP@?$AAB?$AAK?$AAL?$AAC?$AAh?$AAa?$AAn?$AAg?$AAe?$AAI?$AAn?$AAC?$AAo?$AAn?$AAt?$AAr?$AAo?$AAl?$AAP?$AAa?$AAn?$AAe?$AAl?$AA?$AA@ 10001178     backlight_common_topaz_v1:backlight.obj
 0001:000001a8       ??_C@_1DE@PFEDGFDL@?$AAB?$AAa?$AAc?$AAk?$AAL?$AAi?$AAg?$AAh?$AAt?$AAL?$AAe?$AAv?$AAe?$AAl?$AAC?$AAh?$AAa?$AAn?$AAg?$AAe?$AAE?$AAv?$AAe?$AAn?$AAt?$AA?$AA@ 100011a8     backlight_common_topaz_v1:backlight.obj
 0001:000001e0       ??_C@_1EG@KHBDFHDI@?$AAP?$AAo?$AAw?$AAe?$AAr?$AAM?$AAa?$AAn?$AAa?$AAg?$AAe?$AAr?$AA?1?$AAU?$AAs?$AAe?$AAr?$AAA?$AAc?$AAt?$AAi?$AAv?$AAi?$AAt?$AAy?$AA_?$AAI?$AAn?$AAa?$AAc?$AAt?$AAi@ 100011e0     backlight_common_topaz_v1:backlight.obj
 0001:00000228       ??_C@_1EC@PPGKBJLE@?$AAP?$AAo?$AAw?$AAe?$AAr?$AAM?$AAa?$AAn?$AAa?$AAg?$AAe?$AAr?$AA?1?$AAU?$AAs?$AAe?$AAr?$AAA?$AAc?$AAt?$AAi?$AAv?$AAi?$AAt?$AAy?$AA_?$AAA?$AAc?$AAt?$AAi?$AAv?$AAe@ 10001228     backlight_common_topaz_v1:backlight.obj
 0001:0000026c       ??_C@_1CK@NJCEAPDJ@?$AAB?$AAa?$AAc?$AAk?$AAL?$AAi?$AAg?$AAh?$AAt?$AAC?$AAh?$AAa?$AAn?$AAg?$AAe?$AAE?$AAv?$AAe?$AAn?$AAt?$AA?$AA@ 1000126c     backlight_common_topaz_v1:backlight.obj
 0001:00000298       ??_C@_19DINFBLAK@?$AAN?$AAa?$AAm?$AAe?$AA?$AA@ 10001298     backlight_common_topaz_v1:backlight.obj
 0001:000002d0       ?BSPBacklightInitialize@@YAXXZ 100012d0 f   bspbacklight.obj
 0001:0000049c       ?BSPBacklightRelease@@YAXXZ 1000149c f   bspbacklight.obj
 0001:000004bc       ?BSPBacklightSetIntensity@@YAXK@Z 100014bc f   bspbacklight.obj
 0001:00000560       ?BSPBacklightEnable@@YAXXZ 10001560 f   bspbacklight.obj
 0001:00000564       BKL_Deinit                 10001564 f   backlight_common_topaz_v1:backlight.obj
 0001:0000060c       BKL_IOControl              1000160c f   backlight_common_topaz_v1:backlight.obj
 0001:00000824       DllEntry                   10001824 f   backlight_common_topaz_v1:backlight.obj
 0001:0000082c       BKL_Open                   1000182c f   backlight_common_topaz_v1:backlight.obj
 0001:00000830       BKL_Close                  10001830 f   backlight_common_topaz_v1:backlight.obj
 0001:00000838       BKL_PowerDown              10001838 f   backlight_common_topaz_v1:backlight.obj
 0001:0000083c       BKL_PowerUp                1000183c f   backlight_common_topaz_v1:backlight.obj
 0001:00000840       BKL_Read                   10001840 f   backlight_common_topaz_v1:backlight.obj
 0001:00000848       BKL_Write                  10001848 f   backlight_common_topaz_v1:backlight.obj
 0001:00000850       BKL_Seek                   10001850 f   backlight_common_topaz_v1:backlight.obj
 0001:00000a98       ?BKL_EventThread@@YAKPAX@Z 10001a98 f   backlight_common_topaz_v1:backlight.obj
 0001:00000cec       BKL_Init                   10001cec f   backlight_common_topaz_v1:backlight.obj
 0001:00000f90       RegCloseKey                10001f90 f   coredll:COREDLL.dll
 0001:00000fa0       RegQueryValueExW           10001fa0 f   coredll:COREDLL.dll
 0001:00000fb0       RegOpenKeyExW              10001fb0 f   coredll:COREDLL.dll
 0001:00000fc0       EventModify                10001fc0 f   coredll:COREDLL.dll
 0001:00000fd0       DeleteCriticalSection      10001fd0 f   coredll:COREDLL.dll
 0001:00000fe0       CloseMsgQueue              10001fe0 f   coredll:COREDLL.dll
 0001:00000ff0       StopPowerNotifications     10001ff0 f   coredll:COREDLL.dll
 0001:00001000       CloseHandle                10002000 f   coredll:COREDLL.dll
 0001:00001010       SetLastError               10002010 f   coredll:COREDLL.dll
 0001:00001020       LeaveCriticalSection       10002020 f   coredll:COREDLL.dll
 0001:00001030       EnterCriticalSection       10002030 f   coredll:COREDLL.dll
 0001:00001040       GetSystemPowerStatusEx2    10002040 f   coredll:COREDLL.dll
 0001:00001050       ReadMsgQueue               10002050 f   coredll:COREDLL.dll
 0001:00001060       DevicePowerNotify          10002060 f   coredll:COREDLL.dll
 0001:00001070       WaitForSingleObject        10002070 f   coredll:COREDLL.dll
 0001:00001080       WaitForMultipleObjects     10002080 f   coredll:COREDLL.dll
 0001:00001090       CeSetThreadPriority        10002090 f   coredll:COREDLL.dll
 0001:000010a0       CreateThread               100020a0 f   coredll:COREDLL.dll
 0001:000010b0       RequestPowerNotifications  100020b0 f   coredll:COREDLL.dll
 0001:000010c0       CreateMsgQueue             100020c0 f   coredll:COREDLL.dll
 0001:000010d0       CreateEventW               100020d0 f   coredll:COREDLL.dll
 0001:000010e0       GetSystemPowerStatusEx     100020e0 f   coredll:COREDLL.dll
 0001:000010f0       InitializeCriticalSection  100020f0 f   coredll:COREDLL.dll
 0001:00001100       MmMapIoSpace               10002100 f   ceddk:CEDDK.dll
 0001:00001110       MmUnmapIoSpace             10002110 f   ceddk:CEDDK.dll
 0001:00001120       DDKGpioWriteDataPin        10002120 f   cspddk:CSPDDK.dll
 0001:00001130       DDKGpioSetConfig           10002130 f   cspddk:CSPDDK.dll
 0001:00001140       DDKIomuxSetPadConfig       10002140 f   cspddk:CSPDDK.dll
 0001:00001150       DDKIomuxSetPinMux          10002150 f   cspddk:CSPDDK.dll
 0001:00001160       _DllEntryCRTStartup        10002160 f   corelib0:pegdentry.obj
 0001:000011a4       __GSHandlerCheckCommon     100021a4 f   corelib0:gshandler.obj
 0001:000011dc       __GSHandlerCheck           100021dc f   corelib0:gshandler.obj
 0001:000011fc       __security_init_cookie     100021fc f   corelib0:seccinit.obj
 0001:00001248       __security_check_cookie    10002248 f   corelib0:armsecgs.obj
 0001:00001258       __gsfailure                10002258     corelib0:armsecgs.obj
 0001:0000135c       _cexit                     1000235c f   corelib0:cexit.obj
 0001:0000136c       _initterm                  1000236c f   corelib0:crt0dat.obj
 0001:00001398       _cinit                     10002398 f   corelib0:crt0dat.obj
 0001:000013f8       __crt_ExitProcess          100023f8 f   corelib0:exitproc_proxy.obj
 0001:00001404       memcpy                     10002404 f   corelib1:COREDLL.dll
 0001:00001414       memset                     10002414 f   corelib1:COREDLL.dll
 0001:00001424       __security_gen_cookie2     10002424 f   corelib1:COREDLL.dll
 0001:00001434       __report_gsfailure         10002434 f   corelib1:COREDLL.dll
 0001:00001444       free                       10002444 f   corelib1:COREDLL.dll
 0001:00001454       TerminateProcess           10002454 f   coredll:COREDLL.dll
 0001:00001468       __IMPORT_DESCRIPTOR_COREDLL 10002468     coredll:COREDLL.dll
 0001:0000147c       __IMPORT_DESCRIPTOR_CEDDK  1000247c     ceddk:CEDDK.dll
 0001:00001490       __IMPORT_DESCRIPTOR_CSPDDK 10002490     cspddk:CSPDDK.dll
 0001:000014a4       __NULL_IMPORT_DESCRIPTOR   100024a4     coredll:COREDLL.dll
 0002:00000000       __imp_MmMapIoSpace         10003000     ceddk:CEDDK.dll
 0002:00000004       __imp_MmUnmapIoSpace       10003004     ceddk:CEDDK.dll
 0002:00000008       \177CEDDK_NULL_THUNK_DATA  10003008     ceddk:CEDDK.dll
 0002:0000000c       __imp_EventModify          1000300c     coredll:COREDLL.dll
 0002:00000010       __imp_DeleteCriticalSection 10003010     coredll:COREDLL.dll
 0002:00000014       __imp_CloseMsgQueue        10003014     coredll:COREDLL.dll
 0002:00000018       __imp_StopPowerNotifications 10003018     coredll:COREDLL.dll
 0002:0000001c       __imp_CloseHandle          1000301c     coredll:COREDLL.dll
 0002:00000020       __imp_SetLastError         10003020     coredll:COREDLL.dll
 0002:00000024       __imp_LeaveCriticalSection 10003024     coredll:COREDLL.dll
 0002:00000028       __imp_EnterCriticalSection 10003028     coredll:COREDLL.dll
 0002:0000002c       __imp_GetSystemPowerStatusEx2 1000302c     coredll:COREDLL.dll
 0002:00000030       __imp_ReadMsgQueue         10003030     coredll:COREDLL.dll
 0002:00000034       __imp_RegOpenKeyExW        10003034     coredll:COREDLL.dll
 0002:00000038       __imp_WaitForSingleObject  10003038     coredll:COREDLL.dll
 0002:0000003c       __imp_WaitForMultipleObjects 1000303c     coredll:COREDLL.dll
 0002:00000040       __imp_CeSetThreadPriority  10003040     coredll:COREDLL.dll
 0002:00000044       __imp_CreateThread         10003044     coredll:COREDLL.dll
 0002:00000048       __imp_RequestPowerNotifications 10003048     coredll:COREDLL.dll
 0002:0000004c       __imp_CreateMsgQueue       1000304c     coredll:COREDLL.dll
 0002:00000050       __imp_CreateEventW         10003050     coredll:COREDLL.dll
 0002:00000054       __imp_GetSystemPowerStatusEx 10003054     coredll:COREDLL.dll
 0002:00000058       __imp_InitializeCriticalSection 10003058     coredll:COREDLL.dll
 0002:0000005c       __imp_RegQueryValueExW     1000305c     coredll:COREDLL.dll
 0002:00000060       __imp_DevicePowerNotify    10003060     coredll:COREDLL.dll
 0002:00000064       __imp_RegCloseKey          10003064     coredll:COREDLL.dll
 0002:00000068       __imp_free                 10003068     corelib1:COREDLL.dll
 0002:0000006c       __imp___report_gsfailure   1000306c     corelib1:COREDLL.dll
 0002:00000070       __imp_memcpy               10003070     corelib1:COREDLL.dll
 0002:00000074       __imp_memset               10003074     corelib1:COREDLL.dll
 0002:00000078       __imp___security_gen_cookie2 10003078     corelib1:COREDLL.dll
 0002:0000007c       __imp_TerminateProcess     1000307c     coredll:COREDLL.dll
 0002:00000080       \177COREDLL_NULL_THUNK_DATA 10003080     coredll:COREDLL.dll
 0002:00000084       __imp_DDKIomuxSetPadConfig 10003084     cspddk:CSPDDK.dll
 0002:00000088       __imp_DDKGpioSetConfig     10003088     cspddk:CSPDDK.dll
 0002:0000008c       __imp_DDKGpioWriteDataPin  1000308c     cspddk:CSPDDK.dll
 0002:00000090       __imp_DDKIomuxSetPinMux    10003090     cspddk:CSPDDK.dll
 0002:00000094       \177CSPDDK_NULL_THUNK_DATA 10003094     cspddk:CSPDDK.dll
 0002:0000012c       __security_cookie          1000312c     corelib0:seccinit.obj
 0002:00000130       __security_cookie_complement 10003130     corelib0:seccinit.obj
 0002:000001c4       _exitflag                  100031c4     corelib0:cexit.obj
 0002:000001c8       __onexitend                100031c8     <common>
 0002:000001cc       __onexitbegin              100031cc     <common>

 entry point at        0001:00001160

 Static symbols

 0001:00000858       ?GetBacklightLevelSettings@@YAXPAU_bklSettings@@@Z 10001858 f   backlight_common_topaz_v1:backlight.obj
 0001:00000948       ?GetBacklightTimeoutSettings@@YAXPAU_bklSettings@@@Z 10001948 f   backlight_common_topaz_v1:backlight.obj
 0001:0000129c       doexit                     1000229c f   corelib0:cexit.obj
